:020000040000FA
:10000000D8A2FF9AA2C886B2208E1DD0FB208E1DDA
:10001000F0FB20F91DC90CD00FA21FB5709550CA76
:1000200010F986DCA9CCD012C90ED00720B202A9E3
:10003000EED007C914D00B20A30385FB85FA85F900
:0F004000D0BEC90FD006204B034C9D014C96013A
:1000700003040007020501061017111612151413C8
:1000800073747077727571766067616662656463B8
:10009000F0FF0110110FEFF1DFE1EEF2120E1F2160
:1000A0000B0A06060404040402020202020202020F
:1000C00099250B25010033250736340D34340E52A3
:0D00D000250D45350455220643330FCC00A5
:10010000A6B5305CA5B0F008E008D004C5E6F02E36
:10011000F6E3C901D002F6E3501EA00FA5B1D960E5
:1001200000F0038810F8B9A000D5E4900494E69597
:10013000E4180875E595E528E004F003303160A582
:10014000E885DDA90085B5204B0320B2022000021E
:1001500020B202A90885B52009022031034C001AFB
:10016000E0F9D00BA560C5B1D004A90085B46050FA
:10017000FDA007A5B1D96000F00588F0F110F6B92F
:10018000A000D5E2900295E2C6B5A9FBC5B5F00383
:10019000202503E6B560C908B01220EB03A21FB505
:0F01A00050C5FAF003CA10F786FB86B04C00007A
:10020000A210A90095DECA10FBA91085B0C6B010D7
:100210000160201E03A4B0A20886B6C0081041C029
:1002200006102EC004101FC001F009100E208E020F
:10023000D0FBF0D9209C02D0FBF0D2A20486B620DD
:100240009C02D0FBF0C7209C02A5B6C904D0F7F0F1
:10025000BCA21086B6208E02A5B6C908D0F7F0ADB4
:10026000A20686B620CA0250053003200001201ED7
:1002700003C6B6A5B6C905F0EB20CA02708F308D53
:10028000200001A5B129F0C920F0EE4C0D0220CAD2
:10029000023003200001201E03C6B66020CA02906F
:1002A0000250F93007082000012850F0201E03C634
:1002B000B660A20F38B460A977F5509560945038B5
:1002C000A977F5509550CA10EB60A5B1A6B6187580
:1002D0008F85B12988D042A5B1A220CA300ED55051
:1002E000D0F9E0103033A97F69017001B8A5B530AD
:1002F00024C90810204808A9F985B585B4204B0306
:1003000020B202200902202E03286885B5A5B4304A
:100310000438A9FF6018A90060A9FF18B860A6B04A
:10032000B55085B160204B0320B20220090220B2F3
:1003300002BA86B3A6B29A6885B66885B0AA6895EF
:100340005068AA6885B195504C7003BA86B3A6B2BE
:100350009AA5B148A8A21FD550F003CA10F9A9CC9C
:1003600095508A48A6B0B5509450488A48A5B648DA
:10037000BA86B2A6B39A60A6E4E4A0D004A900F0BD
:100380000AA6E3D006A6EED002A9FFA20486B5C550
:10039000FA900CF00A85FAA5B085FBA5B185F92085
:1003A0008E1D60A6DC1017A5F9D5DCD00FCAB5DC10
:1003B00085FBCAB5DC85F9CA86DCD01A85DCA20CBF
:1003C00086B586FAA214200202A20486B520000295
:1003D000A6FAE00F9012A6FBB55085FA86B0A5F9F3
:1003E00085B1204B034C0000A9FF60A20406F9264A
:0B03F000FACAD0F905F985F985B16063
:101A000018A98065EB65EC65ED65E165DF38E5F00B
:101A1000E5F1E5E2E5E0E5DEE5EFE5E3B002A900AA
:101A20004A18694065EC65ED38E5E44A1869906547
:101A3000DD65DD65DD65DD65E138E5E4E5E4E5E529
:101A4000E5E5E5E0A6B1E033F016E034F012E0227F
:101A5000F00EE025F00AA6B0F009B450C010100353
:061A60001869024C770337
:00000001FF
